:100000000C9464000C948C000C948C000C948C0068
:100010000C948C000C948C000C948C000C948C0030
:100020000C948C000C948C000C948C000C948C0020
:100030000C948C000C948C000C948C000C948C0010
:100040000C94A10D0C948C000C9411100C948C0049
:100050000C948C000C948C000C948C000C948C00F0
:100060000C948C000C948C000000000024002700ED
:100070002A0000000000250028002B0000000000DE
:1000800023002600290004040404040404040202DA
:100090000202020203030303030301020408102007
:1000A0004080010204081020010204081020000012
:1000B0000007000201000003040600000000000029
:1000C00000008F00750B971111241FBECFEFD8E0F1
:1000D000DEBFCDBF12E0A0E0B1E0E0E3F5E402C096
:1000E00005900D92AA3DB107D9F713E0AAEDB2E051
:1000F00001C01D92AF3AB107E1F710E0C8ECD0E0C3
:1001000004C02297FE010E942C22C23CD107C9F7ED
:100110000E940C010C9496220C94000008951092F9
:10012000DB021092DC021092DD028AED92E09093E5
:10013000DF028093DE021092E0021092E20210923F
:10014000E1028CE061E00E94400F8CE06091DB02F4
:100150000E94660F08958F929F92BF92CF92DF9276
:10016000EF92FF920F931F93CF93DF936B01C09198
:10017000E502D091E6022197B090E7027C01EC0EF7
:10018000FD1E00E010E08FEF882E912C36C0F701A5
:100190007081802F033010F060E005C060E0F1E076
:1001A000FB1508F461E0833010F490E005C090E0A6
:1001B00023E0B21609F491E0F801EE5DFE4F808174
:1001C000292F30E040E050E0662311F041E050E09C
:1001D000242B352B672F70E0232B21F0F401E61B35
:1001E000F70BBF010E94E00E0F5F1F4F219608948E
:1001F000E11CF11C0630110519F0CC15DD0538F2B3
:10020000DF91CF911F910F91FF90EF90DF90CF90F2
:10021000BF909F908F900895EF92FF920F931F933E
:10022000DF93CF9300D000D0CDB7DEB70E94800E11
:1002300085EE92E00E94540DE090E70200E010E0AD
:10024000F801EE5DFE4FF0808F2D61E00E94400FBF
:10025000802F033010F040E005C040E091E09E1593
:1002600008F441E0833010F480E005C080E093E0C2
:10027000E91609F481E090E020E030E0442311F039
:1002800021E030E0822B932B892B19F460E070E0A1
:1002900002C06FEF70E08F2D0E94E00E0F5F1F4FC6
:1002A0000630110569F68DE061E00E94400F8DE097
:1002B0006091E3020E94660F8E010F5F1F4FC8011D
:1002C00068E072E046E751E00E94160BC8010E9408
:1002D000950A80E090E00F900F900F900F90CF91D3
:1002E000DF911F910F91FF90EF90089585EE92E0BE
:1002F0000E94FE0B882319F081E08093DC020895B0
:10030000CF92DF92EF92FF920F931F9385EE92E0D0
:100310000E94A50C8C013AEDC32E32E0D32EC6010B
:100320006DE440E150E00E94380B27E9E22E23E023
:10033000F22EC701602F0E948411012F110F110BA3
:10034000C701602F0E948411C70163E171E04EE094
:1003500050E00E94E911C6010E94320B1F910F91DB
:10036000FF90EF90DF90CF900895EF92FF920F9360
:100370001F934AEDE42E42E0F42EC7016EE444E1FF
:1003800050E00E94380B07E913E0C8016DE271E00C
:1003900042E050E00E94E911C80160E071E042E1F2
:1003A00050E00E94E911C7010E94320B1F910F918A
:1003B000FF90EF9008950F931F93DF93CF9300D09A
:1003C00000D0CDB7DEB785EE92E00E94990C69832C
:1003D0007A838B839C830AED12E0C8016AE044E0D3
:1003E00050E00E94380B87E993E0BE016F5F7F4FBA
:1003F00044E050E00E94E911C8010E94320B0F90C6
:100400000F900F900F90CF91DF911F910F91089552
:100410000F931F93CF93DF93EB018A018A3069F129
:100420008B3030F4833059F0863009F040C011C071
:100430008E3431F1823551F18D34C9F524C08AED05
:1004400092E063E045E050E028E231E00E945A0B80
:100450002EC08881882359F560E08091E3028823CB
:1004600009F461E06093E3028DE00E94660FCE0123
:100470000196B8010E94AB001AC00E94DB0117C0B0
:100480000E94B50114C00E94800111C060E08091FB
:10049000E302882309F461E06093E3028DE00E94A7
:1004A000660F8BED92E0BE01A8010E949D02DF91D4
:1004B000CF911F910F910895F999FECF72BD61BD43
:1004C000F89A80B50895F999FECF1FBA72BD61BD43
:1004D00040BD0FB6F894FA9AF99A0FBE0895CF93DB
:1004E000DF93EB01A0E0B0E020E030E0425050406C
:1004F00008C0FE01E20FF31F8081A80FB11D2F5F1E
:100500003F4F24173507ACF38A812B2F3327FE0189
:10051000E80FF11D808190E02817390711F020E0E5
:1005200008C020E0B070818190E0A817B90709F4F5
:1005300021E0822FDF91CF910895EF92FF920F93E8
:100540001F93CF93DF938C01EB014A31510574F077
:1005500088818C3C59F48981813041F48A8190E012
:100560009A01225030408217930721F0C801039668
:1005700062E0F5C0C8010E946F02882321F4C8011F
:10058000039663E0ECC0FF24F39445E050E02F2D88
:1005900030E060E070E0FE01E40FF51F80818F3FE6
:1005A00011F461E070E026233723FF24232B11F0A0
:1005B000FF24F3944F5F5F4F4930510541F7FF200F
:1005C000A1F4BE016D5F7F4F85EE92E00E94100D99
:1005D000882309F4C1C0BE016B5F7F4F85EE92E0B6
:1005E0000E94E30C882309F4B7C0EC8820E2E216ED
:1005F00041F080E3E81629F0C801039665E00E9407
:1006000077099A8980E02B89AC01420F511DCA01FC
:1006100001978E5F9F4F38F4C80103966F2DAE018E
:1006200029E030E079C09D8980E02E89BC01620F0D
:10063000711DAFE2B1E0E0E0F0E020E030E08D914C
:100640009C9111978617970759F4F901EE0FFF1F38
:10065000E20FF31FEE0FFF1FEE0FFF1FE15DFE4FD6
:100660002F5F3F4F1C962431310549F7309739F4FD
:10067000C80103966F2DAE0120E030E04DC080E24E
:10068000E816E9F582819381892B19F4848180FF32
:100690003DC0FF2021F0C801039661E060C0452BFA
:1006A00031F0C8010396BE0149E050E009C09F89BE
:1006B0008285981741F0C8010396BE0141E050E0E1
:1006C0000E94470A4EC0848195812281338180FF38
:1006D0000EC0FC01F595E795E00FF11F0190F08148
:1006E000E02DE20FF31F0190F081E02D01C0F90130
:1006F00095958795800F911FBE01099532C086811F
:100700009781892B61F4808580FD09C0C80103961B
:100710006F2DAE0125E030E00E945F0A22C0808587
:1007200091852681378180FF0EC0FC01F595E79504
:10073000E00FF11F0190F081E02DE20FF31F019017
:10074000F081E02D01C0F90195958795800F911FEB
:100750006F2D9E01099505C0C801039664E00E94B3
:100760007709DF91CF911F910F91FF90EF9008953E
:10077000FF920F931F93CF93DF938C01F62EE90125
:100780008F89843031F0C8010396A90121E030E05F
:1007900021C0F90140E050E060E070E090E0762F89
:1007A000652F542F4427808D480F511D611D711DE9
:1007B0009F5F3196943099F74F3F8FEF58078FEF37
:1007C00068078FEF780749F4C80103966F2DAE01D3
:1007D00026E030E00E945F0A0FC085EE92E00E94A2
:1007E000D20BC8010396FF2021F061E00E94770937
:1007F00003C0BE010E94880ADF91CF911F910F9123
:10080000FF900895DC01F9018789823031F0CD0134
:100810000396A90121E030E017C020E030E0808D90
:10082000853611F421E030E040E050E0818D8E36D5
:1008300011F441E050E024233523232B41F4CD0172
:100840000396AF0126E030E00E945F0A0895CD01D3
:100850000396662321F061E00E9477090895BF01A5
:100860000E94880A0895FF920F931F93CF93DF93FE
:10087000EC01F62E8901F9018789813031F0CE0132
:100880000396A90121E030E00AC0F901608D6230D1
:1008900048F0CE0103966F2DA90126E030E00E94BA
:1008A0005F0A11C0611161E068838CE00E94660FED
:1008B000CE010396FF2021F061E00E94770903C07A
:1008C000B8010E94880ADF91CF911F910F91FF908C
:1008D0000895FF920F931F93CF93DF938C01F62E11
:1008E000E9018F89843041F0C8010396A90121E014
:1008F00030E00E945F0A22C0F90140E050E060E071
:1009000070E090E0762F652F542F4427808D480F9C
:10091000511D611D711D9F5F3196943099F785EED1
:1009200092E00E94C50BC8010396FF2021F061E010
:100930000E94770903C0BE010E94880ADF91CF910F
:100940001F910F91FF900895FF920F931F93CF93E4
:10095000DF938C01F62EE9018F89823031F0C801D6
:100960000396A90121E030E013C0988D80E0298D25
:10097000BC01620F711D6115710521F082E06130CB
:1009800078074CF0C80103966F2DAE0126E030E0E9
:100990000E945F0A0FC085EE92E00E94EB0BC80137
:1009A0000396FF2021F061E00E94770903C0BE0199
:1009B0000E94880ADF91CF911F910F91FF900895B7
:1009C000FF920F931F93CF93DF938C01F62EE901D3
:1009D0008F89813031F0C8010396A90121E030E010
:1009E0000BC0688D862F8150833048F0C801039674
:1009F0006F2DA90126E030E00E945F0A0FC085EE4E
:100A000092E00E94230CC8010396FF2021F061E0D0
:100A10000E94770903C0BE010E94880ADF91CF912E
:100A20001F910F91FF900895DF92EF92FF920F9325
:100A30001F93CF93DF937C01D62E8901F90147895B
:100A4000413238F00396A90121E030E00E945F0AAC
:100A50001CC0B901685E7F4F85EE92E00E943D0D9B
:100A6000E7012396DD2029F0CE0161E00E9477099D
:100A70000CC0CE01B80144E050E00E946A0A81E057
:100A8000F7018183CE010E940F09DF91CF911F9161
:100A90000F91FF90EF90DF900895EF92FF920F93E8
:100AA0001F937C018C010D5F1F4FC80141E050E096
:100AB0000E94820AC801F70160810E943A09C801B8
:100AC0000E941D091F910F91FF90EF9008950F93C1
:100AD0001F938C010D5F1F4FC80142E050E00E9440
:100AE000820AC8016091E7020E943A09C80163E0E6
:100AF0000E943A09C8010E941D091F910F91089593
:100B00000F931F938C010D5F1F4FC80144E050E00D
:100B10000E94820AC80161E30E943A09C8016EE29C
:100B20000E943A09C80160E30E943A09C80160E0E6
:100B30000E943A09C8010E941D091F910F91089552
:100B4000AF92BF92CF92DF92EF92FF920F931F93DB
:100B50008C015B0185EE92E00E94810C6B017C01AF
:100B60000D5F1F4FC801B50144E050E00E94820AAA
:100B7000C801B701A6010E945B09C8010E941D09B6
:100B80001F910F91FF90EF90DF90CF90BF90AF90AB
:100B900008950F931F93CF93DF93EB01288D8C0162
:100BA0000D5F1F4F222331F0C80146E050E00E9444
:100BB000470A3AC0C8014DE150E00E94820AC801CC
:100BC000688D0E943A09C80160E00E943A09C80194
:100BD00061E00E943A09C80161E00E943A09C80137
:100BE00060E070E00E944609C8016CED75E00E946B
:100BF0004609C80164E670E00E944609C80160E940
:100C000071E00E944609C80161E00E943A09C3E709
:100C1000D2E0C80169910E943A0982E0C338D8073E
:100C2000C1F7C8010E941D09DF91CF911F910F915B
:100C30000895EF92FF920F931F93E090E502F090DA
:100C4000E6028C010D5F1F4FC80142E050E00E9498
:100C5000820AC801B7010E944609C8010E941D0905
:100C60001F910F91FF90EF9008950F931F938C01A8
:100C70000D5F1F4FC80142E050E00E94820AC80188
:100C800063E074E00E944609C8010E941D091F919B
:100C90000F910895FF920F931F938C010D5F1F4FCB
:100CA000C80143E150E00E94820AC80160E071E09F
:100CB0000E944609C80162E070E00E944609C8012E
:100CC00068E075E00E944609C80141E050E060E03C
:100CD00070E00E945B09F090E702EF2DF0E0EE0F6C
:100CE000FF1FEE0FFF1FE65BFD4F6181C80170E043
:100CF0000E944609C8016F2D0E943A09C80163E0AD
:100D00000E943A096091E5027091E602C8010E94D2
:100D10004609C80160E070E00E944609C80161E030
:100D20000E943A09C8010E941D091F910F91FF906E
:100D300008950F931F93CF93DF93FB01308D20E035
:100D4000418D240F311D8C010D5F1F4F2050304805
:100D500031F0C80146E050E00E94470A44C0C80193
:100D600045E250E00E94820AC80160E070E80E94FB
:100D70004609C80164E00E943A09C80163E00E9484
:100D80003A09C80162E00E943A09C80160E00E9485
:100D90003A09C80160E00E943A09C80160E00E9477
:100DA0003A09C80140E050E060E070E00E945B0951
:100DB000C8014EEF5FEF6FEF7FEF0E945B09C80144
:100DC00041E050E060E070E00E945B09C1E6D2E0E3
:100DD000C80169910E943A0982E0C237D807C1F779
:100DE000C8010E941D09DF91CF911F910F910895B5
:100DF0000F931F93CF93DF939C01EAE3F1E040E070
:100E0000808181114F5F3C9682E0EA32F807C1F79A
:100E100089010D5F1F4F50E0440F551FC8010E940C
:100E2000820ACFE2D1E08B85882329F0688179811D
:100E3000C8010E9446092C9682E0CF31D80799F765
:100E4000C8010E941D09DF91CF911F910F91089554
:100E50009F92AF92BF92CF92DF92EF92FF920F9349
:100E60001F93CF93DF93DB0158969C90589799205E
:100E700019F023E0291538F40396BD0146E050E04F
:100E80000E94470A3FC0092D10E001501040000F9A
:100E9000111F000F111FF801E05BFD4FA080B18012
:100EA000E50109900020E9F77E010894E108F108C6
:100EB000EA18FB0823E0C22ED12CC80ED91EA701C8
:100EC0004D5F5F4FC6010E94820AC601692D0E94D4
:100ED0003A09025B1D4FF8016181C60170E00E9472
:100EE0004609C0E0D0E008C0F501EC0FFD1FC601C7
:100EF00060810E943A092196CE15DF05A8F3C6014C
:100F00000E941D09DF91CF911F910F91FF90EF90EB
:100F1000DF90CF90BF90AF909F900895EF92FF9297
:100F20000F931F93CF93DF93EC017B01898188237B
:100F300059F08E010D5F1F4FC8010E9416091982DA
:100F400081E08A83C80109C08A81882381F0FB017E
:100F5000808D813061F4CE010396B70140E050E00E
:100F600020E030E001E3F2E8EF2EF12C0CC01A8211
:100F7000CE010396B70140E050E020E030E001E20E
:100F8000E0E3EE2EF12C0E949209CE0103960E941E
:100F90001D09DF91CF911F910F91FF90EF90089560
:100FA000CF92DF92EF92FF920F931F93CF93DF9335
:100FB0006A018C010D5F1F4FE22EFF24C80140E043
:100FC00050E097010E94270AC0E0D0E008C0F60177
:100FD000EC0FFD1FC80160810E943A092196CE15D1
:100FE000DF05A8F3C8010E941D09DF91CF911F9171
:100FF0000F91FF90EF90DF90CF9008954AE552E077
:1010000022E00E94D0070895CF92DF92EF92FF92E4
:101010000F931F93DF93CF93CDB7DEB7A0970FB693
:10102000F894DEBF0FBECDBF7C016B0185EE92E070
:101030008E010F5F1F4FB80140E20E94AA0C282FBB
:10104000C701B601A8010E94D007A0960FB6F89478
:10105000DEBF0FBECDBFCF91DF911F910F91FF90EB
:10106000EF90DF90CF90089543E151E0209121016E
:101070000E94D007089540E051E0209112010E94A3
:10108000D007089580E00E94BE0EAA2797FDA09584
:10109000BA2FBC01CD010E94DA2020E030E048E404
:1010A00052E40E948A2120E030E048EC52E40E94A1
:1010B0008A2120E030E040E85AE30E948A210E9421
:1010C000A720CB010895FF920F931F93CF93DF9337
:1010D000EC01F62E8901F9018789813031F0CE01CA
:1010E0000396A90121E030E00AC0F901808D81500A
:1010F0008E3F40F4CE010396A90126E030E00E9425
:101100005F0A13C0CE010E944208BC0185EE92E046
:101110000E94DF0BCE010396FF2021F061E00E94C8
:10112000770903C0B8010E94880ADF91CF911F910F
:101130000F91FF900895CF92DF92EF92FF920F935D
:101140001F936C017B018C010D5F1F4FC80149E0AB
:1011500050E00E94820AC801F701608D0E943A099E
:10116000C6010E944208BC01C8010E944609C8018C
:1011700060E070E00E944609C80160E070E00E94F3
:10118000460985EE92E00E94A00CBC01C8010E94B5
:101190004609C8010E941D091F910F91FF90EF9011
:1011A000DF90CF9008950F931F93CF93DF938C011F
:1011B000E9018F89813041F0C8010396A90121E03E
:1011C00030E00E945F0A16C0888D81508E3F40F447
:1011D000C8010396B90146E050E00E94470A0AC0E0
:1011E00085EE92E060E070E00E94DF0BC801BE0176
:1011F0000E949B08DF91CF911F910F9108959C0150
:10120000FB01808D882339F0C901039646E050E048
:101210000E94470A0895C9010E949B080895FC0195
:1012200082818F3F11F08F5F82830895FC0182815C
:10123000882311F0815082830895EF92FF920F93DB
:101240001F938C0187E9E82E83E0F82EF801648172
:10125000C7010E948411C701F80163810E948411B3
:10126000F801808191810E94320B1F910F91FF90B4
:10127000EF900895FC0183819481860F911D9483E2
:10128000838387E993E00E9484110895EF92FF928F
:101290000F931F938C017B01672F770F770BC8018A
:1012A0000E943A09C8016E2D0E943A091F910F91C0
:1012B000FF90EF900895CF92DF92EF92FF920F93FD
:1012C0001F936C017A018B019B01552737FD5095C7
:1012D000452FB9010E944609C601B7010E9446097F
:1012E0001F910F91FF90EF90DF90CF900895FF92A4
:1012F0000F931F938C01F62EFC018081918162E592
:1013000041E050E00E94380B87E993E06F2D0E9486
:101310008411F801808191810E94320B1F910F91FD
:10132000FF9008956F927F928F929F92AF92BF929B
:10133000CF92DF92EF92FF920F931F936C015B01AC
:10134000142F3901FC0114821382A901455E5F4FFD
:101350008081918162E50E94380BC60160E00E94A5
:101360003A09C6016CEC0E943A09C60161E00E948C
:101370003A09662D685EC6010E943A09C601F50168
:1013800061850E943A09C601F50162850E943A0909
:10139000C601F50163850E943A09C601F50164851D
:1013A0000E943A09C601F50165850E943A09C60105
:1013B000F50166850E943A0945EE842E42E0942E9E
:1013C000C4010E94A50CBC01C6010E944609C401CB
:1013D0000E94990CAB01BC01C6010E945B09C601C9
:1013E000F50167850E943A09C601612F0E943A09FA
:1013F000C601F60162810E943A09C601F5016289BF
:101400000E943A09C601F50163890E943A09C601A2
:10141000602F0E943A096F2D772767FD7A95C601E4
:101420000E943A09C6016E2D0E943A09C601662D36
:101430000E943A091F910F91FF90EF90DF90CF909B
:10144000BF90AF909F908F907F906F900895EF9294
:10145000FF920F937C01DB0155969C915597569610
:101460006C91569754968C915497803211F001E309
:1014700001C001E2F92FE0E0E60FF11DC701BD0157
:101480007F010E9492090F91FF90EF900895EF92D3
:10149000FF920F931F938C017A0142E050E022E00B
:1014A00030E00E94270AC801B7010E944609C8011E
:1014B0000E941D091F910F91FF90EF9008956623E0
:1014C00021F061E00E9477090895BA01A9010E9404
:1014D000470A0895EF92FF920F931F938C017A01B0
:1014E00041E050E022E030E00E94270AC801B70145
:1014F0000E944609C8010E941D091F910F91FF908B
:10150000EF9008959A0140E050E00E94270A089564
:101510000F931F938C0140E050E00E94820AC801A3
:101520000E941D091F910F9108955F926F927F9203
:101530008F929F92AF92BF92CF92DF92EF92FF92E3
:101540000F931F93DF93CF93CDB7DEB7C855D2402B
:101550000FB6F894DEBF0FBECDBF4C0100E010E027
:101560005524EE24FF24CC24DD243E010894611C84
:10157000711C06C0D4011296ED91FC911397099548
:1015800087E993E00E942911892BA1F387E993E071
:101590000E94541102301105E9F0033011053CF4AA
:1015A0000115110591F00130110551F70AC0043001
:1015B000110509F104301105A4F00530110501F7FA
:1015C00029C0582E02E010E0DBCF8E37C9F601E0CB
:1015D00010E0D6CFE82EFF2403E010E0CC24DD2479
:1015E000CFCFB82EAA24EA0CFB1CE114F10479F049
:1015F00004E010E0C5CFF301EC0DFD1D80830894DD
:10160000C11CD11CCE14DF0409F0BACF760105E06D
:1016100010E0B6CF873E39F4D401ED91FC91852DD1
:10162000B301A701099500E010E0AACFFC01718386
:1016300060835383428387E993E040E052EC61E0AA
:1016400070E00E94A2100895FC01718360835383AF
:10165000428387E993E040E052EC61E070E00E9451
:10166000A210089587E993E067EE0E94841108951F
:10167000DF92EF92FF920F931F93D62E7A0107E924
:1016800013E0C8016EE70E948411C8016D2D0E940D
:101690008411C8016E2D0E948411EF2CFF0CFF08ED
:1016A000C8016E2D0E9484111F910F91FF90EF9041
:1016B000DF900895CF92DF92EF92FF920F931F93E6
:1016C0006C018A0179010E94380B87E993E0B70128
:1016D000A8010E94E911C6010E94320B1F910F91CF
:1016E000FF90EF90DF90CF90089510920803109232
:1016F00009030895CF92DF92EF92FF920F931F9309
:101700008B016A0194EEE92E92E0F92E452F550FD8
:10171000550BC7010E9463020F5F1F4FC701B8013D
:101720004C2D0E9463021F910F91FF90EF90DF906C
:10173000CF9008958F929F92AF92BF92CF92DF92F7
:10174000EF92FF920F931F934C01580169017A01A8
:101750008601332717FD3095232FBA01A8010E9477
:101760007A0B82E090E0E80EF91EC401B701A501F2
:101770000E947A0B1F910F91FF90EF90DF90CF9016
:10178000BF90AF909F908F9008950F931F938A0101
:101790009B014CE250E060E070E00E949A0B1F91C8
:1017A0000F9108950F931F938A019B0146E050E02B
:1017B00060E070E00E949A0B1F910F910895AB01B9
:1017C0006EE270E00E947A0B0895AB0164E070E075
:1017D0000E947A0B0895EF92FF920F931F937C0162
:1017E0008B0162E070E0A8010E947A0BF70111837F
:1017F00000831F910F91FF90EF9008951F93CF9357
:10180000DF93EC018BA18823D1F010E00DC0612F94
:1018100070E0FE01E60FF71F84EE92E0645F7F4FF9
:1018200043810E9463021F5F4CA1141780F3CE0115
:101830006AE070E050E00E947A0B1BA281E0DF9129
:10184000CF911F910895FF920F931F938C01F62E55
:1018500084EE92E060E370E04F2D0E946302F80195
:10186000F2821F910F91FF900895DF92EF92FF9205
:101870000F931F938B0134EEE32E32E0F32EC7015A
:101880000E945C02D82E0F5F1F4FC701B8010E9453
:101890005C023D2D20E0280F311DC9011F910F91E1
:1018A000FF90EF90DF900895AF92BF92CF92DF92BA
:1018B000EF92FF920F931F935C016A01BA010E949D
:1018C000350C7C0100E010E08701FF24EE2482E06B
:1018D00090E0C80ED91EC501B6010E94350C9C01CE
:1018E00040E050E02E0D3F1D401F511FB901CA01BD
:1018F0001F910F91FF90EF90DF90CF90BF90AF902E
:1019000008954CE250E060E070E00E94540C0895AD
:101910000F931F938C010E94810CAB01BC014F5FA0
:101920005F4F6F4F7F4FC8010E94C50B1F910F91F2
:10193000089546E050E060E070E00E94540C089585
:101940006EE270E00E94350C089564E070E00E9441
:10195000350C0895EF92FF920F931F93CF93DF936F
:10196000EC01062FF72E142F6AE070E00E94350C70
:10197000212F30E08217930710F0E12E06C0CE0130
:101980006AE070E00E94350CE82E802F9F2D9C01AC
:101990008901C0E0D0E00CC02C9684EE92E0BE013C
:1019A0000E945C02F80181938F012B97882319F024
:1019B000FC2ECE1588F38F2DDF91CF911F910F91C3
:1019C000FF90EF900895FF920F931F93CF93DF93B3
:1019D0008B01FF24F394C6E0D0E084EE92E0BE01D8
:1019E0000E945C0220E030E0F8019081891711F438
:1019F00021E030E08F2D90E028233923FF24232B92
:101A000011F0FF24F39421960F5F1F4FCA30D105C8
:101A100021F78F2DDF91CF911F910F91FF900895A6
:101A2000FF920F931F93CF93DF938B01FF24F394C7
:101A3000C4E0D0E084EE92E0BE010E945C0220E0AF
:101A400030E0F8019081891711F421E030E08F2D0A
:101A500090E028233923FF24232B11F0FF24F39453
:101A600021960F5F1F4FC830D10521F78F2DDF91D1
:101A7000CF911F910F91FF9008951F93CF93DF9304
:101A8000EC01142F413208F010E29E012D5F3F4F10
:101A9000C901412F50E00E94C61E1CA381E08BA308
:101AA000DF91CF911F910895CF93DF93EC0160E018
:101AB00070E00E94350C8D549F4479F1CE0160E0B6
:101AC00070E04DE45FE40E947A0BCE0161E070E0CB
:101AD0000E94EB0BCE0160E77AE70E94E50BCE0196
:101AE00041E050E060E070E00E94D20BCE016AE875
:101AF00072E04EE00E943D0DCE0140E050E060E01B
:101B000070E00E94C50BCE0160E070E00E94DF0B28
:101B1000CE0161E00E94230C0EC0CE0162E070E0B5
:101B20000E94350C9983888384EE92E060E370E034
:101B30000E945C028A83CE010E94880CDF91CF91C3
:101B400008951F920F920FB60F9211242F933F9377
:101B50008F939F93AF93BF9380910E0390910F0348
:101B6000A0911003B0911103309112030196A11DB1
:101B7000B11D232F2D5F2D3720F02D570196A11D6C
:101B8000B11D2093120380930E0390930F03A09333
:101B90001003B093110380910A0390910B03A0915D
:101BA0000C03B0910D030196A11DB11D80930A0392
:101BB00090930B03A0930C03B0930D03BF91AF91CF
:101BC0009F918F913F912F910F900FBE0F901F907B
:101BD00018958FB7F89420910E0330910F03409120
:101BE0001003509111038FBFB901CA0108959FB727
:101BF000F89420910A0330910B0340910C0350910B
:101C00000D0386B5A89B06C08F3F21F02F5F3F4F85
:101C10004F4F5F4F9FBF542F432F322F2227280F44
:101C2000311D411D511D82E0220F331F441F551FDE
:101C30008A95D1F7B901CA0108959B01AC017FB71C
:101C4000F89480910A0390910B03A0910C03B0913A
:101C50000D0366B5A89B05C06F3F19F00196A11D45
:101C6000B11D7FBFBA2FA92F982F8827860F911DEE
:101C7000A11DB11D62E0880F991FAA1FBB1F6A95A5
:101C8000D1F7BC012DC0FFB7F89480910A03909161
:101C90000B03A0910C03B0910D03E6B5A89B05C002
:101CA000EF3F19F00196A11DB11DFFBFBA2FA92F5B
:101CB000982F88278E0F911DA11DB11DE2E0880F7E
:101CC000991FAA1FBB1FEA95D1F7861B970B885E49
:101CD0009340C8F2215030404040504068517C4F02
:101CE000211531054105510571F60895019739F027
:101CF000880F991F880F991F02970197F1F7089590
:101D0000789484B5826084BD84B5816084BD85B5D6
:101D1000826085BD85B5816085BDEEE6F0E080819D
:101D200081608083E1E8F0E01082808182608083BE
:101D3000808181608083E0E8F0E080818160808341
:101D4000E1EBF0E0808184608083E0EBF0E0808173
:101D500081608083EAE7F0E0808184608083808115
:101D600082608083808181608083808180688083BD
:101D70001092C10008958093A1020895982F8E308B
:101D800008F09E5097708091A1028295880F880F6D
:101D9000807C892B80937C0080917A008064809382
:101DA0007A0080917A0086FDFCCF209178004091E6
:101DB0007900942F80E030E0282B392BC901089559
:101DC0001F93CF93DF93182FEB0161E00E94400F28
:101DD000209709F44AC0CF3FD10509F449C0E12F4B
:101DE000F0E0E255FF4F84918330C1F0843028F455
:101DF000813051F08230B1F50CC0863019F1873056
:101E000049F1843079F514C084B5806884BDC7BDBC
:101E100033C084B5806284BDC8BD2EC0809180006F
:101E2000806880938000D0938900C093880024C08C
:101E300080918000806280938000D0938B00C0935B
:101E40008A001AC08091B00080688093B000C0936F
:101E5000B30012C08091B00080628093B000C09344
:101E6000B4000AC0C038D1051CF4812F60E002C064
:101E7000812F61E00E94660FDF91CF911F9108953D
:101E8000482F50E0CA0186569F4FFC0124914A57C3
:101E90005F4FFA0184918823C1F0E82FF0E0EE0F44
:101EA000FF1FE859FF4FA591B491662341F49FB7F6
:101EB000F8948C91209582238C939FBF08959FB7AF
:101EC000F8948C91822B8C939FBF0895482F50E0FB
:101ED000CA0182559F4FFC012491CA0186569F4F2B
:101EE000FC0134914A575F4FFA019491992309F408
:101EF00044C0222351F1233071F0243028F42130E2
:101F0000A1F0223011F514C02630B1F02730C1F015
:101F10002430D9F404C0809180008F7703C0809171
:101F200080008F7D8093800010C084B58F7702C0C1
:101F300084B58F7D84BD09C08091B0008F7703C0C8
:101F40008091B0008F7D8093B000E92FF0E0EE0F1C
:101F5000FF1FEE58FF4FA591B491662341F49FB740
:101F6000F8948C91309583238C939FBF08959FB7ED
:101F7000F8948C91832B8C939FBF0895682F70E009
:101F8000CB0182559F4FFC012491CB0186569F4F78
:101F9000FC0144916A577F4FFB019491992319F4F6
:101FA00020E030E03CC0222351F1233071F0243096
:101FB00028F42130A1F0223011F514C02630B1F000
:101FC0002730C1F02430D9F404C0809180008F778D
:101FD00003C0809180008F7D8093800010C084B505
:101FE0008F7702C084B58F7D84BD09C08091B00019
:101FF0008F7703C08091B0008F7D8093B000892FD0
:1020000090E0880F991F84589F4FFC01A591B491CF
:102010008C9120E030E0842311F021E030E0C90110
:1020200008951F920F920FB60F9211242F933F9392
:102030004F938F939F93EF93FF934091C600E0914E
:102040009303F091940331969F012F77307031976D
:1020500080919503909196032817390739F0ED5E2A
:10206000FC4F40833093940320939303FF91EF91AF
:102070009F918F914F913F912F910F900FBE0F9095
:102080001F9018958F92AF92CF92DF92EF92FF92AE
:102090000F931F93DF93CF93CDB7DEB7FC0186EA92
:1020A00092E0918380837383628355834483378373
:1020B000268311870087F386E286D586C486A686A6
:1020C00087868D85808B8E85818B8F85828BCF9146
:1020D000DF911F910F91FF90EF90DF90CF90AF9025
:1020E0008F9008958F92AF92CF92DF92EF92FF92EE
:1020F0000F931F93DF93CF93CDB7DEB7FC0186EA32
:1021000092E0918380837383628355834483378312
:10211000268311870087F386E286D586C486A68645
:1021200087868D85808B8E85818B8F85828BCF91E5
:10213000DF911F910F91FF90EF90DF90CF90AF90C4
:102140008F900895CF93DF93EC019A01AB01E8855E
:10215000F985203081EE380780E0480780E0580795
:1021600009F449C081E090E00A8802C0880F991FF5
:102170000A94E2F7808360E079E08DE390E00E94CA
:102180000F222150304040405040CA01B90122E0A6
:1021900030E040E050E00E940F22EC81FD8130836E
:1021A000EE81FF812083EA85FB85208141E050E0BC
:1021B000CA010E8402C0880F991F0A94E2F7282BE7
:1021C0002083EA85FB852081CA010F8402C0880F25
:1021D000991F0A94E2F7282B2083EA85FB858081EA
:1021E000088802C0440F551F0A94E2F7842B8083AD
:1021F000DF91CF910895108220E130E0CECFFC0135
:10220000A285B3854C9121E030E0C901068402C06B
:10221000880F991F0A94E2F7809584238C93A285F6
:10222000B3854C91C901078402C0880F991F0A9495
:10223000E2F7809584238C93A285B3858C910088E6
:1022400002C0220F331F0A94E2F7209528232C9313
:102250000895DC011296ED91FC911397E058FF4F21
:102260002191319180819181281B390B2F7730701A
:10227000C9010895DC011296ED91FC911397EE5778
:10228000FF4F2081318192918291E058F040821776
:10229000930719F42FEF3FEF05C0E20FF31F808182
:1022A000282F30E0C9010895DC011296ED91FC91D0
:1022B0001397DF01AE57BF4F2D913C911197E05816
:1022C000FF4F80819181E058F0408217930719F405
:1022D0002FEF3FEF0BC0E20FF31F80812F5F3F4FC7
:1022E0002F7730702D933C93282F30E0C90108954B
:1022F000DC011296ED91FC911397EE57FF4F808110
:102300009181929382930895FC01A085B1852189E2
:102310008C9190E0022E02C0959587950A94E2F781
:1023200080FFF6CF0484F585E02D6083089586EA6A
:1023300092E0909398038093970383E193E09093C6
:102340009A038093990385EC90E090939C0380938B
:102350009B0384EC90E090939E0380939D0380EC1C
:1023600090E09093A00380939F0381EC90E0909382
:10237000A2038093A10386EC90E09093A403809342
:10238000A30384E08093A50383E08093A60387E002
:102390008093A70385E08093A80381E08093A9033D
:1023A00008950F931F93CF93DF938C01EB0109C026
:1023B0002196D801ED91FC910190F081E02DC801AA
:1023C000099568816623A1F7DF91CF911F910F9145
:1023D0000895EF92FF920F931F93CF93DF938C0199
:1023E0007B01EA010CC0D7016D917D01D801ED910F
:1023F000FC910190F081E02DC8010995219720976B
:1024000091F7DF91CF911F910F91FF90EF90089579
:10241000DC01ED91FC910280F381E02D0995089596
:10242000CF92DF92EF92FF920F931F93CF93DF93A0
:102430006C017B01C0E0D0E00EC0D601ED91FC91B3
:1024400000811181C701BE010E94D814682FC60106
:10245000F80109952196F70184819581C817D9075C
:1024600060F3DF91CF911F910F91FF90EF90DF907C
:10247000CF9008952F923F924F925F926F927F92EA
:102480008F929F92AF92BF92CF92DF92EF92FF9284
:102490000F931F93DF93CF93CDB7DEB7A0970FB6FF
:1024A000F894DEBF0FBECDBF1C016A017B01411550
:1024B00051056105710549F440E350E060E070E0CA
:1024C00020E030E00E94061356C08824992454016D
:1024D000422E55246624772401E010E00C0F1D1FC6
:1024E000080D191DC701B601A30192010E94ED213B
:1024F000F80160830894811C911CA11CB11CC701C8
:10250000B601A30192010E94ED21C901DA016C011B
:102510007D01C114D104E104F104F1F681E0E82E5B
:10252000F12CEC0EFD1EE80CF91C3E010894611C18
:10253000711CD501C4010197A109B1096C01C8182A
:10254000D90816C0F601EE0DFF1D40814A3010F487
:10255000405D01C0495C552747FD5095652F752F9B
:10256000C10120E030E00E9406130894E108F10860
:102570006E147F0439F7A0960FB6F894DEBF0FBE35
:10258000CDBFCF91DF911F910F91FF90EF90DF9022
:10259000CF90BF90AF909F908F907F906F905F9003
:1025A0004F903F902F900895DC012115310541F4A3
:1025B000ED91FC910190F081E02D642F0995089533
:1025C0000E943A120895EF92FF920F931F939A017F
:1025D0007B0100E010E0B801A7010E94D4121F9116
:1025E0000F91FF90EF900895EF92FF920F931F933A
:1025F0009A01E62EFF2400E010E0B801A7010E9436
:10260000D4121F910F91FF90EF900895EF92FF92D7
:102610000F931F93CF93DF93EC017A018B01211568
:10262000310541F4E881F9810190F081E02D642FBA
:1026300009951BC02A303105B1F477FF10C04DE277
:1026400050E060E070E020E030E00E94061310955A
:102650000095F094E094E11CF11C011D111DCE01C8
:10266000B801A7012AE00E943A12DF91CF911F9191
:102670000F91FF90EF900895EF92FF920F931F93A9
:102680007B019A010027F7FC0095102FB801A701E4
:102690000E9406131F910F91FF90EF900895EF9203
:1026A000FF920F931F93E62E9A01FF24E7FCF0940C
:1026B0000F2D1F2DB801A7010E9406131F910F9126
:1026C000FF90EF9008950F931F938C014DE050E021
:1026D00060E070E020E030E00E940613C8014AE0AC
:1026E00050E060E070E020E030E00E9406131F91AF
:1026F0000F9108950F931F938C010E94D412C8016B
:102700000E9463131F910F910895CF92DF92EF9271
:10271000FF920F931F938C019A016B01EE24FF240B
:10272000B701A6010E94D412C8010E9463131F9131
:102730000F91FF90EF90DF90CF900895CF92DF92AE
:10274000EF92FF920F931F938C019A01C62EDD2406
:10275000EE24FF24B701A6010E94D412C8010E94F2
:1027600063131F910F91FF90EF90DF90CF9008952A
:102770000F931F938C010E940812C8010E946313DB
:102780001F910F9108950F931F938C010E941012B7
:10279000C8010E9463131F910F9108950F931F9317
:1027A0008C010E940613C8010E9463131F910F91B0
:1027B0000895CF92DF92EF92FF920F931F938C01B7
:1027C0006B019A01EE24D7FCE094FE2CB701A60120
:1027D0000E940613C8010E9463131F910F91FF907E
:1027E000EF90DF90CF900895CF92DF92EF92FF921B
:1027F0000F931F938C01C62E9A01DD24C7FCD09441
:10280000ED2CFD2CB701A6010E940613C8010E9401
:1028100063131F910F91FF90EF90DF90CF90089579
:102820009F92AF92BF92CF92DF92EF92FF920F935F
:102830001F93CF93DF93EC017A018B01922ECB0192
:10284000BA0120E030E040E050E00E943B208823C5
:102850006CF4CE014DE250E060E070E020E030E04A
:102860000E94061317FB109517F9109520E030E031
:1028700040E05FE3AA240BC0CA01B90120E030E0C8
:1028800040E251E40E943F209B01AC01A394A914B3
:1028900098F3C801B7010E94D71F5B016C010E9429
:1028A000AC207B018C01CE01B801A7012AE030E009
:1028B0000E94D412992029F0CE0166EC72E00E94A9
:1028C0000812C801B7010E94D8209B01AC01C601C3
:1028D000B5010E94D61F22C020E030E040E251E462
:1028E0000E948A217B018C010E94A7205B016C0160
:1028F000CC24B7FCC094DC2CCE01B601A5012AE0A3
:1029000030E00E940613C601B5010E94DA209B0147
:10291000AC01C801B7010E94D61F9A949920E1F634
:10292000DF91CF911F910F91FF90EF90DF90CF90AB
:10293000BF90AF909F9008950E94101408950F9338
:102940001F938C010E941014C8010E9463131F91F1
:102950000F910895FC010190F081E02DE60FF71F23
:1029600080810895DC01ED91FC911197309751F031
:1029700014968D919C9115976817790718F4E60FB6
:10298000F71F40830895FC019B018481958168179E
:10299000790728F4608171816115710529F410921D
:1029A000AA036AEA73E002C0620F731FCB010895A5
:1029B000FC010190F081E02DE60FF71F8081089562
:1029C000FC01808191810E949F1E08950F931F93A7
:1029D000CF93DF93FC018B0141155105A1F06115E7
:1029E000710589F084819581EA0121978C179D07F3
:1029F00008F4EC0160817181C801AE010E94031FDF
:102A0000C00FD11F1882DF91CF911F910F910895B0
:102A10000F931F93CF93DF93FC018B014115510559
:102A2000A1F06115710589F084819581EA012197F2
:102A30008C179D0708F4EC0160817181C801AE011B
:102A40000E94031FC00FD11F1882DF91CF911F91E9
:102A50000F9108950F931F938C01FC018081918148
:102A60000E94721DF80113821282158214821F9136
:102A70000F910895FC01DB0114962D913C9115975F
:102A800084819581821B930B8417950710F480E055
:102A90000895808191816D917C91840F951FA9018A
:102AA0000E94F51E9C0180E0232B09F481E008952B
:102AB000FC01DB012481358114968D919C91159741
:102AC0002817390710F480E00895CF0140E050E066
:102AD0000E943A150895DF92EF92FF920F931F9391
:102AE000CF93DF93EC018C819D8148175907C8F47F
:102AF0007A010894E11CF11CE881F981EE0DFF1DBB
:102B0000D080108208811981772767FD7095C801F0
:102B10000E94121F9C010E0D1F1DF801D08200970C
:102B200019F4EFEFFFEF05C088819981F901E81BE7
:102B3000F90BCF01DF91CF911F910F91FF90EF9093
:102B4000DF900895FC0144815581415050400E941E
:102B50006B150895CF93DF93FC01DB018481958190
:102B60004817590760F4C081D1816D917C91CE01E5
:102B7000840F951F0E941D1F9C01009719F42FEFD1
:102B80003FEF02C02C1B3D0BC901DF91CF9108958F
:102B900040E050E00E94AA150895CF93DF93FC0116
:102BA000848195814817590768F4C081D1817727BE
:102BB00067FD7095CE01840F951F0E94DA1E9C015F
:102BC000009719F42FEF3FEF02C02C1B3D0BC901FA
:102BD000DF91CF91089540E050E00E94CD15089517
:102BE000DC01FB0114962D913C9115978481958110
:102BF0002817390711F080E00895608171818D9167
:102C00009C910E94E51E9C0180E0232B09F481E049
:102C10000895FC01DB012481358114968D919C91EE
:102C200015972817390710F480E00895281B390BF1
:102C3000808191816D917C91820F931F0E94E51E8E
:102C40009C0180E0232B09F481E00895DC01FB0165
:102C5000608171818D919C910E94E51E292F3327FF
:102C600027FD3095209530952227330F221F3327DB
:102C7000C9010895DC01FB01608171818D919C91F6
:102C80000E94E51E40E050E01816190614F041E0DD
:102C900050E0CA010895DC01FB01608171818D91D2
:102CA0009C910E94E51E40E050E01816190614F4AD
:102CB00041E050E0CA010895DC01FB0160817181AF
:102CC0008D919C910E94E51E292F332727FD309579
:102CD0002227330F221F3327C9010895DC01FB018E
:102CE00014962D913C911597848195812817390769
:102CF00051F4608171818D919C910E94E51E9C012F
:102D000080E0232B09F081E090E00895DC01FB01D5
:102D100014962D913C911597848195812817390738
:102D200011F080E00BC0608171818D919C910E94B7
:102D3000E51E9C0180E0232B09F481E090E00895DA
:102D4000FC01DB016D917C91808191810E94E51EE7
:102D500008950F931F93CF93DF93EC018B01FB0139
:102D6000648175818C819D81680F791F7D836C835F
:102D70008A819B8186179707B8F46F5F7F4F8881A0
:102D800099810E94CA1D4C815D81009729F0998329
:102D900088835B834A8308C0F80184819581481B3E
:102DA000590B5D834C8307C0F80160817181888174
:102DB00099810E94CF1ECE01DF91CF911F910F917B
:102DC00008950E94A9160895CF93DF93EC01CB01DB
:102DD0007B836A8301960E94C81C9983888300972D
:102DE00021F41B821A821D821C82DF91CF910895EB
:102DF0000F931F93CF93DF93EC018B0186179707F7
:102E000009F1FB01248135818C819D818217930713
:102E100050F4888199810E94721DF8016481758146
:102E2000CE010E94E416288139812115310551F027
:102E3000F801848195819D838C8360817181C901B2
:102E40000E94EE1ECE01DF91CF911F910F91089548
:102E50001F93CF93DF93EC01162F81E090E09D83C9
:102E60008C83CE0161E070E00E94E416E881F98174
:102E7000309721F01083E881F9811182DF91CF91A1
:102E80001F9108951F93CF93DF93EC01162F81E0DC
:102E900090E09D838C83CE0161E070E00E94E41697
:102EA000E881F981309721F01083E881F98111825E
:102EB000DF91CF911F9108951F93CF93DF93EC0182
:102EC000162F81E090E09D838C83CE0161E070E05D
:102ED0000E94E416E881F981309721F01083E8819F
:102EE000F9811182DF91CF911F9108951F93CF93A4
:102EF000DF93EC01162F81E090E09D838C83CE015F
:102F000061E070E00E94E416E881F981309721F0D9
:102F10001083E881F9811182DF91CF911F9108958B
:102F20000F931F93CF93DF938C01EB016C817D8115
:102F3000FC01758364830E94E416F801808191810D
:102F4000009721F0688179810E94EE1EDF91CF9178
:102F50001F910F9108950F931F93CF93DF938C01CF
:102F6000EB016C817D81FC01758364830E94E41612
:102F7000F80180819181009721F0688179810E9418
:102F8000EE1EDF91CF911F910F910895EF92FF9266
:102F90000F931F93DF93CF93CDB7DEB7A1970FB6F3
:102FA000F894DEBF0FBECDBF8C01CB01BA017E010C
:102FB0000894E11CF11CA7012AE030E00E94A11F47
:102FC000F70101900020E9F73197EE19FF09D801C8
:102FD0001596FC93EE931497C801BF010E94E41666
:102FE000F80180819181009719F0B7010E94EE1ECF
:102FF000A1960FB6F894DEBF0FBECDBFCF91DF9183
:103000001F910F91FF90EF900895EF92FF920F9311
:103010001F93DF93CF93CDB7DEB7A1970FB6F89488
:10302000DEBF0FBECDBF8C01CB01BA017E0108947B
:10303000E11CF11CA7012AE030E00E94A11FF7016A
:1030400001900020E9F73197EE19FF09D801159694
:10305000FC93EE931497C801BF010E94E416F80197
:1030600080819181009719F0B7010E94EE1EA19610
:103070000FB6F894DEBF0FBECDBFCF91DF911F9189
:103080000F91FF90EF900895EF92FF920F931F938F
:10309000DF93CF93CDB7DEB7A1970FB6F894DEBF1D
:1030A0000FBECDBF8C019A0180E090E07E010894B4
:1030B000E11CF11CA7010E94A11FF7010190002053
:1030C000E9F73197EE19FF09D8011596FC93EE93B5
:1030D0001497C801BF010E94E416F8018081918114
:1030E000009719F0B7010E94EE1EA1960FB6F89452
:1030F000DEBF0FBECDBFCF91DF911F910F91FF902B
:10310000EF900895EF92FF920F931F93DF93CF9369
:10311000CDB7DEB7A1970FB6F894DEBF0FBECDBF17
:103120008C019A0180E090E07E010894E11CF11C82
:10313000A7010E94A11FF70101900020E9F7319734
:10314000EE19FF09D8011596FC93EE931497C80168
:10315000BF010E94E416F80180819181009719F067
:10316000B7010E94EE1EA1960FB6F894DEBF0FBE07
:10317000CDBFCF91DF911F910F91FF90EF900895F8
:103180000F931F93CF93DF938C01EB0161157105B2
:1031900011F4C2EDD2E0FE0101900020E9F7319771
:1031A000EC1BFD0BD8011596FC93EE931497C80108
:1031B000BF010E94E416F80180819181009719F007
:1031C000BE010E94EE1EDF91CF911F910F910895D5
:1031D000AF92BF92CF92DF92EF92FF920F931F9325
:1031E000CF93DF93B82EA92E6B01C82FD92FFB01E7
:1031F00060817181CE010E94C018EE24FF2410C0AE
:10320000088119810E0D1F1DF8018081992787FD06
:1032100090950E944022F80180830894E11CF11CE3
:10322000F60184819581E816F90650F38B2D9A2DCD
:10323000DF91CF911F910F91FF90EF90DF90CF9092
:10324000BF90AF900895AF92BF92CF92DF92EF926E
:10325000FF920F931F93CF93DF93B82EA92E6B018C
:10326000C82FD92FFB0160817181CE010E94C01847
:10327000EE24FF2410C0088119810E0D1F1DF801D6
:103280008081992787FD90950E943822F8018083DC
:103290000894E11CF11CF60184819581E816F90679
:1032A00050F38B2D9A2DDF91CF911F910F91FF90AD
:1032B000EF90DF90CF90BF90AF900895EF92FF9284
:1032C0000F931F93DF93CF93CDB7DEB72C970FB635
:1032D000F894DEBF0FBECDBFFC017B0186179707B8
:1032E00011F401E029C024813581DB0114968D9110
:1032F0009C9115972817390711F000E01DC0CE01E9
:103300000196BF010E94231909811A81CE010796F7
:10331000B7010E9423196F817885C8010E94E51EBC
:1033200000E0009709F401E0CE0107960E942A15FB
:10333000CE0101960E942A15802F2C960FB6F89484
:10334000DEBF0FBECDBFCF91DF911F910F91FF90D8
:10335000EF900895CF92DF92EF92FF921F93CF9359
:10336000DF936C017B01B9012417350710F4BA0112
:10337000A901D70114968D919C911597EB018617A1
:10338000970708F4EC01D701ED91FC911197EC0F30
:10339000FD1F108110826D917C91640F751FC60115
:1033A0000E94C018D701ED91FC91EC0FFD1F108316
:1033B000C601DF91CF911F91FF90EF90DF90CF90EA
:1033C00008950F931F938C01FB01248135810E9486
:1033D000AA19C8011F910F9108958F929F92AF92E1
:1033E000BF92CF92DF92EF92FF920F931F93DF93E2
:1033F000CF9300D000D000D0CDB7DEB75C016B0119
:10340000DB0114968D919C9115970097A1F101977E
:103410004817590780F1F5018481958148175907AC
:1034200050F5ED91FC9100817A014E010894811CC8
:10343000911C1FC0D501ED91FC91EE0DFF1D808107
:103440008017A1F4F601248135812E0D3F1DC401A2
:10345000B501A7010E94AA19C401B6010E94F01586
:10346000182FC4010E942A15112341F40894E10881
:10347000F108F7FEDFCFEE24EA94FE2CC701269672
:103480000FB6F894DEBF0FBECDBFCF91DF911F9175
:103490000F91FF90EF90DF90CF90BF90AF909F90F3
:1034A0008F900895FC01DB014481558114968D9124
:1034B0009C911597481B590BCF010E94ED19089557
:1034C000AF92BF92CF92DF92EF92FF920F931F9332
:1034D000DF93CF9300D000D000D0CDB7DEB75C0132
:1034E0008B01DB016D917C916115710521F4B801AF
:1034F0000E94901742C0CE0101960E94C018F801A8
:10350000E480F580CC24DD2410C0D801ED91FC913D
:10351000EC0DFD1D8081992787FD90950E9430223A
:10352000892B31F00894C11CD11CCE14DF0468F340
:10353000ED80FE800DC0D801ED91FC91EE0DFF1DD8
:103540008081992787FD90950E943022892B31F048
:103550000894E108F108CE14DF0468F30894E11C34
:10356000F11CC5018E010F5F1F4FB801A601970125
:103570000E94AA19C8010E942A15C50126960FB6F5
:10358000F894DEBF0FBECDBFCF91DF911F910F9199
:10359000FF90EF90DF90CF90BF90AF9008952F9263
:1035A0003F924F925F926F927F928F929F92AF92D3
:1035B000BF92CF92DF92EF92FF920F931F93DF9310
:1035C000CF93CDB7DEB768970FB6F894DEBF0FBEC6
:1035D000CDBF3C01FB012A01190160817181611598
:1035E000710521F4BF010E9490175AC07E01089412
:1035F000E11CF11CC7010E94C0188E01095F1F4F1A
:10360000C80162ED72E00E94C018D02EC12E3DE0CC
:10361000832E912C8C0E9D1E23E1A22EB12CAC0E7C
:10362000BD1E24C0C401B70140E050E098010E94D3
:10363000AA198D2D9C2DB4010E94A916C4010E94C7
:103640002A158D2D9C2DB1010E94A916F2014481ED
:103650005581400F511FC501B7010E94E119C701F3
:10366000B5010E94F816C5010E942A15C701B201D2
:103670000E94C8158C01FFEF8F3F9F0799F68D2D93
:103680009C2DB7010E94A916C3016D2D7C2D0E94AF
:1036900090178D2D9C2D0E942A15C7010E942A1576
:1036A000C30168960FB6F894DEBF0FBECDBFCF91B1
:1036B000DF911F910F91FF90EF90DF90CF90BF901F
:1036C000AF909F908F907F906F905F904F903F90C2
:1036D0002F900895DF92EF92FF920F931F93DF9345
:1036E000CF9300D000D000D0CDB7DEB77C01FB0176
:1036F000142FD22E608171816115710521F4BF01F3
:103700000E9490171CC0CE0101960E94C0188981AA
:103710009A81012F112707FD109501C0D082B801B1
:103720000E94DA1EFC010097C9F7C7018E010F5FE6
:103730001F4FB8010E949017C8010E942A15C701A7
:1037400026960FB6F894DEBF0FBECDBFCF91DF91A6
:103750001F910F91FF90EF90DF9008950F931F93AB
:10376000CF93DF938C01EB016115710511F4C2ED6C
:10377000D2E0FE0101900020E9F73197EC1BFD0B30
:10378000D8011596FC93EE931497C801BF010E94CF
:10379000E416F80180819181009719F0BE010E9422
:1037A000EE1EDF91CF911F910F910895EF92FF923E
:1037B0000F931F93DF93CF93CDB7DEB7A1970FB6CB
:1037C000F894DEBF0FBECDBF8C01CB01BA017E01E4
:1037D0000894E11CF11CA7010E94581FF7010190F9
:1037E0000020E9F73197EE19FF09D8011596FC93EF
:1037F000EE931497C801BF010E94E416F80180817E
:103800009181009719F0B7010E94EE1EA1960FB6A4
:10381000F894DEBF0FBECDBFCF91DF911F910F9106
:10382000FF90EF900895EF92FF920F931F93DF9315
:10383000CF93CDB7DEB7A1970FB6F894DEBF0FBE1A
:10384000CDBF8C01CB01BA017E010894E11CF11CB3
:10385000A7010E94581FF70101900020E9F7319756
:10386000EE19FF09D8011596FC93EE931497C80141
:10387000BF010E94E416F80180819181009719F040
:10388000B7010E94EE1EA1960FB6F894DEBF0FBEE0
:10389000CDBFCF91DF911F910F91FF90EF900895D1
:1038A000EF92FF920F931F93DF93CF93CDB7DEB7C5
:1038B000A1970FB6F894DEBF0FBECDBF8C01CB0130
:1038C0007E010894E11CF11CB7010E94371FF7012B
:1038D00001900020E9F73197EE19FF09D8011596FC
:1038E000FC93EE931497C801BF010E94E416F801FF
:1038F00080819181009719F0B7010E94EE1EA19678
:103900000FB6F894DEBF0FBECDBFCF91DF911F91F0
:103910000F91FF90EF900895EF92FF920F931F93F6
:10392000DF93CF93CDB7DEB7A1970FB6F894DEBF84
:103930000FBECDBF8C01CB017E010894E11CF11CB0
:10394000B7010E94371FF70101900020E9F7319776
:10395000EE19FF09D8011596FC93EE931497C80150
:10396000BF010E94E416F80180819181009719F04F
:10397000B7010E94EE1EA1960FB6F894DEBF0FBEEF
:10398000CDBFCF91DF911F910F91FF90EF900895E0
:10399000CF93DF93BC018230910510F462E070E0B8
:1039A000A091AD03B091AE03ED01E0E0F0E040E0A6
:1039B00050E021C0888199818617970769F48A8130
:1039C0009B81309719F09383828304C09093AE0358
:1039D0008093AD03FE0134C06817790738F44115B0
:1039E000510519F08417950708F4AC01FE018A818E
:1039F0009B819C01E9012097E9F641155105A9F148
:103A0000CA01861B970B049708F4BA01E0E0F0E0C6
:103A10002AC08D919C91119784179507F9F464172A
:103A2000750781F412968D919C911397309719F038
:103A30009383828304C09093AE038093AD03FD0112
:103A400032964CC0CA01861B970BFD01E80FF91F87
:103A50006193719302978D939C9340C0FD01828185
:103A600093819C01D9011097A1F68091AB039091AD
:103A7000AC03892B41F48091D5029091D6029093AA
:103A8000AC038093AB034091D7025091D80241150B
:103A9000510541F44DB75EB78091D3029091D402A5
:103AA000481B590B2091AB033091AC03CA01821B18
:103AB000930B8617970780F0AB014E5F5F4F84171B
:103AC000950750F0420F531F5093AC034093AB0344
:103AD000F9016193719302C0E0E0F0E0CF01DF9162
:103AE000CF910895CF93DF93009709F450C0EC0174
:103AF00022971B821A82A091AD03B091AE0310975A
:103B000009F140E050E0AC17BD0708F1BB83AA8380
:103B1000FE0121913191E20FF31FAE17BF0779F437
:103B20008D919C911197280F391F2E5F3F4F39833C
:103B3000288312968D919C9113979B838A834115BC
:103B4000510571F4D093AE03C093AD0320C012961B
:103B50008D919C911397AD01009711F0DC01D3CFAB
:103B6000FA01D383C28321913191E20FF31FCE1763
:103B7000DF0769F488819981280F391F2E5F3F4F35
:103B8000FA01318320838A819B8193838283DF9131
:103B9000CF910895A0E0B0E0E0EDFDE10C9461224A
:103BA0006C01009729F4CB010E94C81C6C01C1C0B4
:103BB0008EEF882E8FEF982E8C0C9D1C8601060FA1
:103BC000171F0815190508F4B2C0F401A081B181CE
:103BD000A617B707B8F0A530B10508F4AAC0CD0103
:103BE00004978617970708F4A4C01297A61BB70B73
:103BF000F801A193B193D4016D937C93CF010E94FE
:103C0000721D97C07B01EA1AFB0AEEEFFFEFEE0E82
:103C1000FF1E36016A0E7B1EC091AD03D091AE032C
:103C200044245524AA24BB244AC0C615D705E1F56F
:103C3000488159814E155F05B8F1CA0104978E1568
:103C40009F05B0F41296A40FB51FF401B183A083B1
:103C50002A813B814114510431F0D20113963C93E7
:103C60002E93129766C03093AE032093AD0361C0CC
:103C70008A819B81F80193838283425050404E1980
:103C80005F09518340834114510431F0D2011396EE
:103C90001C930E93129704C01093AE030093AD03D0
:103CA000F4017183608345C088819981A816B906A3
:103CB00008F45C012E018A819B819C01E901209717
:103CC00009F0B3CF8091AB039091AC0386159705B3
:103CD000E9F4A616B706D0F42091D7023091D802A5
:103CE0002115310541F42DB73EB78091D302909153
:103CF000D402281B390B02171307C8F41093AC0326
:103D00000093AB03D4016D937C9313C0CB010E944D
:103D1000C81CEC01009759F0F40140815181B601B3
:103D20000E94C61EC6010E94721D6E0102C0CC24F4
:103D3000DD24C601CDB7DEB7E0E10C947D221F93F0
:103D4000FC0199278827BC01E89411911032E9F30E
:103D5000193010F01E30C8F31B3251F01D3249F4F7
:103D6000689406C00E948C1F610F711D811D911DFA
:103D7000119110531A30B0F33EF4909580957095E0
:103D800061957F4F8F4F9F4F1F910895FB01DC017D
:103D900002C001900D9241505040D8F70895FB01A8
:103DA000DC010D900020E9F7119701900D920020A1
:103DB000E1F70895FC018191861721F08823D9F756
:103DC000992708953197CF010895FB01DC018D916A
:103DD000019080190110D9F3990B0895FB01DC01C2
:103DE00001900D920020E1F70895FB01DC014150A4
:103DF000504030F08D910190801919F40020B9F7EE
:103E0000881B990B0895FB01DC014150504048F09C
:103E100001900D920020C9F701C01D924150504001
:103E2000E0F70895FC0181E090E00190061609F4A6
:103E3000CF010020D1F701970895FB01519155233F
:103E4000A9F0BF01DC014D9145174111E1F759F48B
:103E5000CD010190002049F04D9140154111C9F369
:103E6000FB014111EFCF81E090E001970895FB0144
:103E70009F01E8944230C4F04532B4F44A3029F44A
:103E800097FB1EF4909581959F4F642F77270E9492
:103E90004B22805D8A330CF0895D8193CB010097C2
:103EA000A1F716F45DE251931082C9010C94C61F6C
:103EB000FA01CF93FF93EF93223044F1253234F58A
:103EC000C22FE894CA3049F497FB3EF49095809550
:103ED000709561957F4F8F4F9F4F2C2F332744272D
:103EE0005527FF93EF930E94ED21EF91FF91605DC5
:103EF0006A330CF0695D6193B901CA01605070408A
:103F00008040904051F716F4CDE2C19310828F911A
:103F10009F91CF910C94C61F592F482F372F262FD2
:103F2000660F771F881F991F660F771F881F991FBD
:103F3000620F731F841F951F660F771F881F991FBD
:103F40000895FA01CF93FF93EF932230CCF02532FE
:103F5000BCF4C22F2C2F332744275527FF93EF9310
:103F60000E94ED21EF91FF91605D6A330CF0695D75
:103F70006193B901CA01605070408040904051F790
:103F800010828F919F91CF910C94C61FDC01FC0190
:103F9000672F71917723E1F7329704C07C916D937D
:103FA00070836291AE17BF07C8F308955058BB27BE
:103FB000AA270ED075C166D130F06BD120F031F454
:103FC0009F3F11F41EF45BC10EF4E095E7FB51C175
:103FD000E92F77D180F3BA17620773078407950733
:103FE00018F071F49EF58FC10EF4E0950B2EBA2FE8
:103FF000A02D0B01B90190010C01CA01A0011124EF
:10400000FF27591B99F0593F50F4503E68F11A169A
:10401000F040A22F232F342F4427585FF3CF46952B
:1040200037952795A795F0405395C9F77EF41F164D
:10403000BA0B620B730B840BBAF09150A1F0FF0F17
:10404000BB1F661F771F881FC2F70EC0BA0F621F03
:10405000731F841F48F4879577956795B795F795F3
:104060009E3F08F0B3CF9395880F08F09927EE0F85
:10407000979587950895D9D008F481E008950CD0DC
:104080000FC107D140F0FED030F021F45F3F19F0AE
:10409000F0C0511139C1F3C014D198F39923C9F379
:1040A0005523B1F3951B550BBB27AA27621773073E
:1040B000840738F09F5F5F4F220F331F441FAA1FF2
:1040C000A9F333D00E2E3AF0E0E830D091505040B2
:1040D000E695001CCAF729D0FE2F27D0660F771F60
:1040E000881FBB1F261737074807AB07B0E809F042
:1040F000BB0B802DBF01FF2793585F4F2AF09E3FD7
:10410000510568F0B6C000C15F3FECF3983EDCF3A8
:10411000869577956795B795F7959F5FC9F7880F4F
:10412000911D9695879597F90895E1E0660F771FA1
:10413000881FBB1F621773078407BA0720F0621B32
:10414000730B840BBA0BEE1F88F7E095089504D02B
:104150006894B111D9C00895BCD088F09F5790F0F1
:10416000B92F9927B751A0F0D1F0660F771F881F9C
:10417000991F1AF0BA95C9F712C0B13081F0C3D0B7
:10418000B1E00895C0C0672F782F8827B85F39F055
:10419000B93FCCF3869577956795B395D9F73EF4FB
:1041A00090958095709561957F4F8F4F9F4F0895A3
:1041B000E89409C097FB3EF49095809570956195C1
:1041C0007F4F8F4F9F4F9923A9F0F92F96E9BB2777
:1041D0009395F695879577956795B795F111F8CFF3
:1041E000FAF4BB0F11F460FF1BC06F5F7F4F8F4F5E
:1041F0009F4F16C0882311F096E911C0772321F054
:104200009EE8872F762F05C0662371F096E8862FEB
:1042100070E060E02AF09A95660F771F881FDAF742
:10422000880F9695879597F90895990F0008550F6F
:10423000AA0BE0E8FEEF16161706E807F907C0F02C
:1042400012161306E407F50798F0621B730B840B34
:10425000950B39F40A2661F0232B242B252B21F40E
:1042600008950A2609F4A140A6958FEF811D811DAE
:10427000089597F99F6780E870E060E008959FEFE8
:1042800080EC089500240A941616170618060906ED
:10429000089500240A9412161306140605060895BC
:1042A000092E0394000C11F4882352F0BB0F40F444
:1042B000BF2B11F460FF04C06F5F7F4F8F4F9F4F84
:1042C000089557FD9058440F551F59F05F3F71F006
:1042D0004795880F97FB991F61F09F3F79F087956D
:1042E0000895121613061406551FF2CF4695F1DFF6
:1042F00008C0161617061806991FF1CF8695710586
:10430000610508940895E894BB2766277727CB01B9
:1043100097F908950BD0C4CFB5DF28F0BADF18F0B5
:10432000952309F0A6CFABCF1124EECFCADFA0F3BF
:10433000959FD1F3950F50E0551F629FF001729F3A
:10434000BB27F00DB11D639FAA27F00DB11DAA1F59
:10435000649F6627B00DA11D661F829F2227B00DA6
:10436000A11D621F739FB00DA11D621F839FA00D31
:10437000611D221F749F3327A00D611D231F849F81
:10438000600D211D822F762F6A2F11249F575040D8
:104390008AF0E1F088234AF0EE0FFF1FBB1F661F73
:1043A000771F881F91505040A9F79E3F510570F02C
:1043B00060CFAACF5F3FECF3983EDCF3869577950C
:1043C0006795B795F795E7959F5FC1F7FE2B880F27
:1043D000911D9695879597F90895A1E21A2EAA1B2B
:1043E000BB1BFD010DC0AA1FBB1FEE1FFF1FA217A5
:1043F000B307E407F50720F0A21BB30BE40BF50BA2
:10440000661F771F881F991F1A9469F7609570952A
:10441000809590959B01AC01BD01CF01089597FB5C
:10442000092E05260ED057FD04D0D7DF0AD0001C78
:1044300038F450954095309521953F4F4F4F5F4F41
:104440000895F6F790958095709561957F4F8F4F01
:104450009F4F0895EE0FFF1F0590F491E02D0994F2
:10446000911116C0803219F089508550D0F7089507
:104470009111089581548A5108F4805E855A0895F7
:104480009111089581568A5108F4805285580895F3
:10449000992788270895AA1BBB1B51E107C0AA1FB3
:1044A000BB1FA617B70710F0A61BB70B881F991FD5
:1044B0005A95A9F780959095BC01CD0108952F924A
:1044C0003F924F925F926F927F928F929F92AF92A4
:1044D000BF92CF92DF92EF92FF920F931F93CF93F1
:1044E000DF93CDB7DEB7CA1BDB0B0FB6F894DEBF88
:1044F0000FBECDBF09942A88398848885F846E84AE
:104500007D848C849B84AA84B984C884DF80EE80F7
:10451000FD800C811B81AA81B981CE0FD11D0FB600
:10452000F894DEBF0FBECDBFED010895F894FFCF24
:1045300041726475696E6F20524742204D697865FB
:104540007200124F70656E204C69676874696E67FF
:10455000000E030506090A0B0001000028010020D7
:10456000008E0700000000000001015000F8060066
:10457000000000000000005100990600000000004B
:1045800000020060004A0600000000000000007009
:10459000003506000000000000000180003B08001C
:1045A000000000000000018100340800000000004D
:1045B000000001820004080000140500000001A0B2
:1045C00000FE070000000000000001B000FE070030
:1045D00000020400000001C000800500000000008F
:1045E000000000E00067050000E00400000001E1B9
:1045F0000028070000000000000101F0001906007B
:1046000000A404000000000002C905000000000032
:104610000001010102FF080000D3080000010102AF
:1046200002000000006308000000010504A005006E
:104630000069040000000100104D05000033040073
:10464000000000008000000000B8030000040136F4
:10465000782050574D00337820696E766572746506
:10466000642050574D2C2033782050574D00367819
:1046700020696E7665727465642050574D0001069E
:104680001F020206260203063E02656E00312E302E
:10469000005365742053657269616C204E756D62BC
:1046A000657200436173652054656D706572617455
:1046B000757265004D4F0100000044656661756CC0
:1046C00074204C6162656C00000204060A0C2C2EFA
:1046D0003001000000008411D111E9112911541199
:1046E0003A117811000000008E00D111E9118E00FE
:1046F0008E008E008E002E00000000008E00D11172
:0A470000E911002000AF03000000E3
:00000001FF
